:0200000480007A
:100000006F000005732F2034930F80006308FF03F7
:10001000930F90006304FF03930FB0006300FF038E
:10002000130F000063040F0067000F00732F2034CC
:1000300063540F006F00400093E19153171F0000BD
:1000400023223FFC171F000023200FFC6FF01FFF2F
:100050009300000013010000930100001302000050
:100060009302000013030000930300001304000038
:100070009304000013050000930500001306000020
:100080009306000013070000930700001308000008
:10009000930800001309000093090000130A0000F0
:1000A000930A0000130B0000930B0000130C0000D8
:1000B000930C0000130D0000930D0000130E0000C0
:1000C000930E0000130F0000930F0000732540F102
:1000D0006310050097020000938202017390523072
:1000E000735044749702000093820201739052305F
:1000F00073500018970200009382020273905230EE
:10010000B70200809382F2FF7390023B9302F001EA
:100110007390023A7350403097020000938242017C
:100120007390523073502030735030309301000080
:1001300097020000938242ED739052301305100035
:100140001315F501634C05000F00F00F930110002B
:100150009308D0051305000073000000930200000F
:10016000638A020073905210B7B20000938292101B
:100170007390223073500030372500007320053013
:100180007350300097020000938242017390123442
:10019000732540F1730020309301200017250000E3
:1001A000130545E6071005008710250007114500D7
:1001B00083166500D371101C538501E4F3151000FC
:1001C000130610006312D5146390C5149301300018
:1001D00017250000130585E307100500871025008B
:1001E0000711450083166500D371101C538501E487
:1001F000F3151000130610006318D5106396C51090
:1002000093014000172500001305C5E00710050005
:10021000871025000711450083166500D371101C57
:10022000538501E4F315100013060000631ED50C7E
:10023000639CC50C9301500017250000130505DED3
:10024000071005008710250007114500831665007B
:10025000D371005C538501E4F31510001306100000
:100260006314D50A6392C50A930160001725000044
:10027000130545DB07100500871025000711450011
:1002800083166500D371005C538501E4F3151000FB
:1002900013060000631AD5066398C5069301700023
:1002A00017250000130585D80710050087102500C5
:1002B0000711450083166500D371005C538501E486
:1002C000F3151000130600016310D504639EC502E8
:1002D00093018000172500001305E5D507100500E0
:1002E000871025000711450083166500D371005C57
:1002F000538501E4F3151000130610006316D500B2
:100300006394C500631030020F00F00F638001009A
:100310009391110093E111009308D005138501001A
:10032000730000000F00F00F930110009308D00538
:0C0330001305000073000000731000C0F3
:1010000000000000000000000000000000000000E0
:1010100000000000000000000000000000000000D0
:1010200000000000000000000000000000000000C0
:1010300000000000000000000000000000000000B0
:081040000000000000000000A8
:102000004842704100009F3CD2E4D3640000FEBB14
:102010004842003C00004842484200000000173F90
:10202000E27000000000405600BC00000000007E8E
:1020300000005859000000008A4A0000000000001B
:040000058000000077
:00000001FF
